:2000000002000812015180FE7581201201A3E58260030200037900E94400601B7A0090012D
:20002000A7780075A000E493F2A308B8000205A0D9F4DAF275A0FFE478FFF6D8FD7800E8E6
:200040004400600A790075A000E4F309D8FC7800E84400600C7900900000E4F0A3D8FCD973
:20006000FA02000385821485831585F016740112016E2514FDE43515FEAF168D828E838FF2
:20008000F0740112016E751702C3E51795135056E5172514FEE43515FFA816A9177A00E99E
:2000A00024FFFBEA34FFFCEB2514FBEC3515FCAD168B828C838DF0120187FBE924FEF9EAD9
:2000C00034FFFAE92514F9EA3515FAAC1689828A838CF0120187F92BFB8E828F8388F012EF
:2000E000016E051780A32285821485831585F016751701751801751902751A03751B057526
:200100001C08751D0D751E15751F227520377D00C3ED95135029ED2514FEE43515FFAA1693
:200120008E828F838AF0120187FE8E80ED2417F886028A90EEB50202800205080D80D1E542
:2001400008600775A0558508B02275A0AA75B0AA2275080075130A90000975F040120064F4
:2001600075130A90000975F0401200E780FE20F71030F6118883A88220F507F6A883758370
:200180000022F280F7F02220F71430F6148883A88220F507E6A88375830022E280F7E49311
:2001A00022E02275820022FFFFFFFFFFFFFFFFFFFFFFFFFFFFFFFFFFFFFFFFFFFFFFFFFF1B
:00000001FF
